:020000020000FC
:100000000CC04AC00000000071C074C07DC0000078
:1000100000000000626B6F3430350FED0DBF00E063
:1000200008BB0CEF07BB08E702BB00E001BB02E026
:1000300003BF02E00EBD772788279927CBD104E6BE
:10004000B02ECAD0C9D0B4D002E3302E06EF202E95
:1000500000E0C02ED02E02EC08BF09BF789403E068
:1000600005BF00E40BBF2AE083FFFECF092D1A2D48
:10007000877F0C541440B8F72A95B1F7F89498D0BC
:1000800097D07894C0E8DBEBC0936B00D0936C0002
:100090000EE100936D00B9C11FB644274BBF45B7B1
:1000A00040FF09C0829B1EC042E045BF4CB55DB514
:1000B000742E852E17C0829915C043E045BF83FD7D
:1000C00011C04CB55DB547195809942EA52E483975
:1000D00068E0560738F4403263E0560718F088604D
:1000E00044E6B42E50E45BBF1FBE18951FB67E7F5A
:1000F0001FBE18951FB67068EE2009F0EA94BB2069
:1001000009F0BA941FBE18951FB676FD2BC040B3F8
:1001100040936F00422D562D541730F43A9459F401
:1001200052E3352E4A9506C031F03A9421F458E254
:10013000352E4395242E706474FF08C094FF03C0CD
:10014000839B72609F7E81FFC69807C075FF03C0C6
:1001500081FFC79802C081FFC598422D4C59409538
:1001600042BF22C0422D42BF7F7B74FF03C080FF8D
:10017000C69A07C075FF03C080FFC79A02C080FF00
:10018000C59A4D3918F482608E7F07C0463F18F03B
:100190008D7F816002C08D7F8E7F86FF05C0C59BED
:1001A00003C0459B74608F7B93FD81601FBE1895D3
:1001B00010E8002702BFC49AC79A02B70032E9F7D5
:1001C000C498C79828E0002702BF02B70F3FE9F79D
:1001D0002A95C9F71A9569F710E828E0002702BFA9
:1001E00002B70F3FE9F72A95C9F71A95B1F70895B5
:1001F00030E03BBF000000000CB51DB508958F7EB8
:1002000083FF14C0092D1A2D877F0C54144010F45D
:1002100000271127169507951695079516950795AA
:10022000202F0456104008F024E6F22F08958F770F
:1002300008958F7D77FF17C07F7772FF06C07B7FA1
:100240004C2D433090F4C39403C0CC2009F0CA94E1
:1002500071FF06C07D7F4D2D443628F4D39403C032
:10026000DD2009F0DA9493D00895F894D6CEC0DF5B
:1002700000936000109361000C0F1D1F32E839BF1E
:100280001BBD0ABD716032EC39BF30E43BBF009149
:10029000640010916500E0916600E695179507955A
:1002A000E695179507952091640030916500E091DF
:1002B0006600201B310BE04000916000109161004E
:1002C000C0916200D09163000093620010936300BC
:1002D0000C1B1D0B200F311F10E0E11F2093640049
:1002E00030936500E09366000895C0916700D09157
:1002F0006800BDDFE69537952795E69537952795F4
:10030000E69537952795E6953795279520936700CD
:10031000309368002093690030936A00089570FD5F
:10032000FECF7160DCE8C0EA63DF0C0F1D1F32E80E
:1003300039BF1BBD0ABD32EC39BF30E43BBF089565
:10034000716056DFC0916900D0916A000C0F1D1FCB
:1003500022E829BF1BBD0ABD22EC29BF30E43BBF08
:1003600084FD4DDF85FD65DF70FDFECF0895C091F2
:100370006B00D0916C007BDF0CB50F70D01BDC38AC
:1003800008F4DBEBD0936C0035D034D008950F2FF8
:100390000D1908F409E095FF05C011E20117B8F046
:1003A000012F15C010916500103438F091609260F3
:1003B00019E1011760F0012F0AC0103238F09E7F5A
:1003C000926012E3011718F0012F01C09C7F009585
:1003D000602E0895F9E006EF202E602E00E008BBA5
:1003E00002E3302E8160977F9062089504E00A95C1
:1003F000F1F7089576FDFECF76FFFECF00916F00F6
:1004000008950895089508950895E4DFFDDFF7DE67
:10041000FA30E8F304E10095602E00EC09BF00001B
:100420007F7D7061C49A81FD02C076FD03C0C798CC
:1004300080FFC69A02EC09BF9B7F00E000936E002C
:1004400004E6E02E94DF05FF12C070FD02C0946048
:1004500016C0D0DFD6DF05FDF8CF00E000936E00B8
:100460000CD10FD11DD1CBDEE2DE81DF36C070FDB5
:1004700002C0946004C0BEDFC4DF05FFF8CFFDD02A
:1004800076DF04FD09C070FD02C094600DC0B2DFCC
:10049000B9DF04FFF8CF08C070FD02C0946004C04B
:1004A000A9DFB0DF04FDF8CFECD0A9DE60DF06FFE6
:1004B00009C070FD02C094600DC09CDFA4DF06FD82
:1004C000F8CF08C070FD02C0946004C093DF9BDFCA
:1004D00006FFF8CFE5D0ABDE4ADF70FD02C09460C6
:1004E00018C088DF8EDF05FFF8CF0BC005FD09C0FF
:1004F00070FD02C094600DC07DDF83DF05FFF8CF83
:1005000008C070FD02C0946004C074DF7ADF05FD8E
:10051000F8CFCAD02CDF04FF09C070FD02C0946080
:100520000DC068DF6FDF04FDF8CF08C070FD02C0AA
:10053000946004C05FDF66DF04FFF8CFC4D079DECB
:1005400016DF06FD09C070FD02C094600DC052DFC9
:100550005ADF06FFF8CF08C070FD02C0946004C0E7
:1005600049DF51DF06FDF8CFB2D0022D063F09F476
:100570004CCFBB2009F47EC0EE2009F47BC0009173
:100580006600002321F400916500043150F00091D1
:100590006E0092FD0027039500936E009B7F0C3345
:1005A00030F00FEFF02EA1DEBCDE9F7D02C0DFDE5B
:1005B0004ACF70FD01C029CF859BFBCF17DF859BFC
:1005C000F8CFBEDE5AD091DEAADE906170FD01C088
:1005D0001CCF8499FBCF0ADF8499F8CF8061B0DE0D
:1005E0009F7E4FD082DE9BDE70FD01C00ECF869BCA
:1005F000FBCFFCDE869BF8CF8068A2DE51D075DE93
:100600008EDE806470FD01C000CF8599FBCFEEDEE9
:100610008599F8CF95DE8F7B47D067DE80DE70FD51
:1006200001C0F3CE849BFBCFE1DE849BF8CF8062D8
:1006300087DE49D05ADE73DE70FD01C0E6CE8699B2
:10064000FBCFD4DE8699F8CF7BDE41D04EDE67DE6D
:10065000BB2081F0022D063F09F4D7CE977FFF2003
:1006600041F0FA9429F00F2D013011F0023009F415
:1006700098609FCFF894AEDED0CCC49880FFC39A28
:10068000089500EC09BF00007F7D7F7E81FD02C0E0
:1006900076FD03C0C69880FFC59A02EC09BF089595
:1006A000C39880FFC29A089500EC09BF00007062F1
:1006B0007F7E81FD02C076FD03C0C59880FFC79A8A
:1006C00002EC09BF0895C29880FFC49A089500EC17
:1006D00009BF00007F7D706181FD02C076FD03C00F
:0C06E000C79880FFC69A02EC09BF08957D
:00000001FF
